:020000020000FC
:10000000D7EED7BBDFEFD8BBEE24552766274424B5
:10001000552466247724442455245527D1E05B7F5A
:10002000B49BFECFB39B5460B499FCCF52FF11C078
:100030005B7FB39905C04D0E5E1CB49BFACF09C01F
:1000400052FF03C044245524F4CF642C752C546013
:10005000F0CF80E0752D2FD181E0742D2CD183E07D
:10006000772D29D184E0762D26D16418750808F4FF
:10007000506486E0752F1FD152FD04C0BDD0BCD0A6
:10008000BBD00BC056FDB8D0F6D0B6D0F4D005C06A
:10009000F2D0B2D0F0D0B0D000C01B2E0A2E412C2E
:1000A000502C612C702CD2E36D0E7E1C4D1A5E0814
:1000B000302E2F2C832C922CA32CB22CDCE3DDE2EF
:1000C000AD0EBE1C8D1A9E08A8956160EE2452FDEF
:1000D00003C092D022D00CC056FD05C0CCD08CD02D
:1000E0001CD008D005C088D0C6D017D003D000C01F
:1000F00063D0EACFCB2DDA2DD01BCF0960F0C92D0C
:10010000D82DD01BCF0938F400C051FF0895577F78
:100110005F7E5D7F089552600895C72DD62DDB1B4D
:10012000CA0B60F1C52DD42DDB1BCA0BB8F500C07E
:100130005E7F4E3118F43E3108F403C04427332764
:100140001CC0433060F053FD07C0222758605F7E1B
:100150005F77C19A442711C0577F44270EC03330C0
:1001600060F054FD07C022275061577F5F77C09A27
:10017000332703C05F7E332700C0089543954E3177
:1001800060F050FD0AC0516057FF02C05F7705C0A4
:1001900050685F7E577F222700C0089533953E3117
:1001A00050F050FD08C0516055FF02C05F7D03C094
:1001B0009927506200C008952395223308F0222722
:1001C0002E3120F000C0C09AC19A08C053FDC098DB
:1001D00054FDC19857FF02C0C098C19855FF09C08F
:1001E0009395933020F0923120F0992704C0C29863
:1001F00002C0C29A00C00895CB2EDA2EBB27AA27D0
:10020000D1E0B49BFECFBD0FAE1DB499FCCF60FF13
:100210000895E12D102DE0581E09DB2FCA2FDE1B9B
:10022000C10B60F0E12D102DD0E8ED0F1E1DDB2F6E
:10023000CA2FDE1BC10B10F4089503C0BC2DAD2DD9
:100240000895CD2DDC2DDB1BCA0B58F0C030B1F763
:10025000C53008F40895AD2DBC2DD5E0BD0FAE1D01
:100260000895CF3F59F7CA3F08F00895AD2DBC2D32
:10027000B550AE090895C02EDF2C0027FF24D1E031
:10028000B39BFECF0D0FFE1CB399FCCF60FF08950A
:10029000E32D122DE0581E09D02FCF2DDE1BC10BF0
:1002A00008F008950C2DFD2C08958EBBE09AE0997E
:1002B000FECF7DB308957DBB8EBBE29AE19AE199B2
:0402C000FECF0895D0
:00000001FF
